:100000000C9435000C945D000C945D000C945D0024
:100010000C945D000C945D000C945D000C945F00EA
:100020000C945D000C945D000C945D000C945D00DC
:100030000C945D000C945D000C945D000C945D00CC
:100040000C9463050C945D000C9432060C945D00D6
:100050000C945D000C945D000C945D000C945D00AC
:100060000C945D000C945D002E0711241FBECFEF91
:10007000D8E0DEBFCDBF11E0A0E0B1E0E8E7F3E1FA
:1000800002C005900D92AC31B107D9F711E0ACE197
:10009000B1E001C01D92AD3FB107E1F710E0CAE643
:1000A000D0E004C02297FE010E943609C836D1076D
:1000B000C9F70E945C050C94BA090C9400001F92C9
:1000C0000F920FB60F921124EF92FF920F931F938E
:1000D0002F933F934F935F936F937F938F939F9350
:1000E000AF93BF93CF93DF93EF93FF9385B18E7D53
:1000F00085B950915C01A7E0B0E0C52FDD27C7FDB1
:10010000D095FD0173E0EE0FFF1F7A95E1F7EC0F3C
:10011000FD1FE45EFE4F9081FD01349763E0EE0F1A
:10012000FF1F6A95E1F7EC0FFD1FE45EFE4F808133
:1001300067E070E0082F10E0E92FF0E029984BB15C
:10014000C801062E02C0880F991F0A94E2F7807832
:100150004F77842B8BB98BB17F01062E02C0EE0C3A
:10016000FF1C0A94E2F797012078307035952795A7
:100170008F7B822B8BB9299A615070408FEF6F3F34
:100180007807E1F61197A330B10509F0BACF85B130
:10019000CC0FDD1FCC0FDD1F837E8C2B85B95F5FFD
:1001A000577050935C0185B1816285B9FF91EF91E1
:1001B000DF91CF91BF91AF919F918F917F916F917F
:1001C0005F914F913F912F911F910F91FF90EF9071
:1001D0000F900FBE0F901F901895089778F477FD39
:1001E0000DC06830710554F457FD08C090E04830E8
:1001F00051050CF091E081E0982701C090E0892F33
:100200000895EF92FF920F931F93CF93DF93F82EF1
:10021000E22E062F10E0C42FD0E090E0B801AE012E
:100220000E94ED00882339F1B801F3E0660F771FD3
:10023000FA95E1F7EE2079F0FB01EC0FFD1FE45E8B
:10024000FE4F208181E090E002C0880F991FFA9450
:10025000E2F7282B0FC0FB01EC0FFD1FE45EFE4F01
:10026000208181E090E002C0880F991FFA94E2F7A4
:10027000809528232083DF91CF911F910F91FF90CC
:10028000EF90089520E030E014C0FC01A3E0EE0FF1
:10029000FF1FAA95E1F7E20FF31FE45EFE4F108205
:1002A00001968830910589F72F5F3F4F283031053F
:1002B00019F080E090E0E9CF0895FF920F931F932B
:1002C000CF93DF93F82EEB018A010E94ED00882383
:1002D000A1F0FE01B3E0EE0FFF1FBA95E1F7E00FCA
:1002E000F11FE45EFE4F208181E090E002C0880FA4
:1002F000991FFA94E2F7282B2083DF91CF911F9169
:100300000F91FF900895FF920F931F93CF93DF9368
:10031000F82EEB018A010E94ED00882389F083E02A
:10032000CC0FDD1F8A95E1F7C00FD11FC45EDE4FF1
:10033000888190E002C095958795FA94E2F78170E4
:10034000DF91CF911F910F91FF900895FF920F932E
:100350001F93CF93DF93F82EEB018A010E94ED00EB
:100360008823A9F0FE0193E0EE0FFF1F9A95E1F7B5
:10037000E00FF11FE45EFE4F208181E090E002C0BB
:10038000880F991FFA94E2F7809528232083DF9144
:10039000CF911F910F91FF9008952130310519F4ED
:1003A0000E945D0108950E94A60108950BC020E0FF
:1003B0000000000000000000000000002F5F2A3550
:1003C000B9F70197009799F7089540E050E010C001
:1003D000FB01E20FF31FE45EFE4F80832F5F3F4F70
:1003E00028303105A9F74F5F5F4F4830510549F07C
:1003F00020E030E0BA01E3E0660F771FEA95E1F70D
:10040000E7CF08959C018830910530F581E090E0B8
:1004100002C0880F991F2A95E2F7982F40E050E01C
:1004200012C0FB01E20FF31FE45EFE4F8081892BB7
:1004300080832F5F3F4F2830310599F74F5F5F4F23
:100440004830510549F020E030E0BA01B3E0660FD2
:10045000771FBA95E1F7E5CF0895823049F08330F0
:10046000F9F08130A1F5862F90E00E9402020895F4
:1004700070E06830710558F520E030E08FEFF90149
:10048000A3E0EE0FFF1FAA95E1F7E60FF71FE45E6A
:10049000FE4F80832F5F3F4F2830310581F708954D
:1004A00070E06830710598F420E030E0E3E0660F1A
:1004B000771FEA95E1F78FEFFB01E20FF31FE45E90
:1004C000FE4F80832F5F3F4F28303105A9F70895F5
:1004D000EF92FF920F931F93E82EF62E072F10E056
:1004E00080E00E94E5018E2D612F0E942D028F2D4C
:1004F000902F0E94D6011F5F183091F717E080E01F
:100500000E94E5018E2D612F0E942D028F2D902FCC
:100510000E94D601115098F71F910F91FF90EF9014
:1005200008954F925F926F927F929F92AF92BF9287
:10053000CF92DF92EF92FF920F931F93CF93DF93AF
:10054000982E162F072F3A0180E00E94E501212FF7
:10055000302FC9016C01C0E0D0E0B7E04B2E512C28
:1005600035C06114710431F0F5018081A201481B8E
:10057000510904C0F7018081482F50E0F3E09F1635
:1005800019F4CE01B8010DC082E0981621F4CE0115
:10059000BA01A80106C091E0991629F4CA01B80170
:1005A000AE010E945D010F5F1F4F0894A11CB11C9A
:1005B0000894E11CF11C0830110599F62196E8E039
:1005C000F0E0CE0EDF1EC830D10529F056017601CD
:1005D00000E010E0C6CFDF91CF911F910F91FF9007
:1005E000EF90DF90CF90BF90AF909F907F906F90F3
:1005F0005F904F900895EF92FF920F931F93CF93C8
:10060000DF9380E00E94E50100E010E08FEEE82E2D
:1006100082E0F82E5DC080E00E94E501CE0165E039
:1006200070E00E949908882777FD8095982F0E9496
:10063000D1058FEF0E94E50164E170E080E090E079
:100640000E94D105CE0166EF7FEF0E94990888EEE7
:1006500093E00E9499086F507040C60FD71F1C1678
:100660001D06CCF264EF71E080E090E00E94D105BD
:10067000CEEED2E080E00E94E501C7018C1B9D0B0D
:1006800065E070E00E949908882777FD8095982F93
:100690000E94D1058FEF0E94E50164E170E080E0E7
:1006A00090E00E94D105CE0166EF7FEF0E9499088D
:1006B00088EE93E00E9499086F507040C60FD71FD4
:1006C0001C161D06BCF20F5F1F4F0230110519F0FA
:1006D000CEEED2E0A0CFDF91CF911F910F91FF908E
:1006E000EF9008952F923F924F925F926F927F9278
:1006F0008F929F92AF92BF92CF92DF92EF92FF9232
:100700000F931F93DF93CF93CDB7DEB7C158D0407F
:100710000FB6F894DEBF0FBECDBFCF57DF4F888333
:10072000C158D0402B013A01490141E4A42EB12C1B
:10073000AC0EBD1EF50131E8C32ED12CCC0EDD1E52
:100740001192EC15FD05E1F700E010E01E010894A0
:10075000211C311C81E088169104C9F414C00E9448
:100760008B0960E470E00E949908E1E4F0E0EC0F8E
:10077000FD1FE80FF91F8081882389F70F5F1F4F46
:1007800091E0908316C0003411054CF312C082E052
:100790008816910471F4003411055CF4E1E4F0E092
:1007A000EC0FFD1FE00FF11F80818F5F80830F5FD3
:1007B0001F4FF501EE24FF249081892F8150863050
:1007C00010F49F5F90838081873019F40894E11CB6
:1007D000F11C3196EC15FD0579F7D101F501808109
:1007E0004114510419F097E0981B892F8C9331968E
:1007F0001196EC15FD0599F7C3010E94D601CF575C
:10080000DF4F8881C158D040B10140E050E00E94E4
:10081000910280E4E816F10409F09CCFCF57DF4F36
:100820000FB6F894DEBF0FBECDBFCF91DF911F9101
:100830000F91FF90EF90DF90CF90BF90AF909F907F
:100840008F907F906F905F904F903F902F90089582
:100850008F929F92AF92BF92CF92DF92EF92FF92D0
:100860000F931F93CF93DF934C018B016130710580
:1008700011F480E001C08FEF0E94E501C0E0D0E0FC
:100880000E948B0968E070E00E949908B82EA92E9A
:100890000E948B0968E070E00E949908D82EC92E4A
:1008A0000E948B0968E070E00E949908F82EE92EFA
:1008B0000115110559F48B2D9A2D6D2D7C2D4F2D81
:1008C0005E2D0E9483018130D9F60DC001301105E3
:1008D000B9F68B2D9A2D6D2D7C2D4F2D5E2D0E94FE
:1008E0008301882369F68B2D9A2D6D2D7C2D4F2D3C
:1008F0005E2D98010E94CD01C4010E94D60121966F
:1009000081E0CF3FD80709F0BBCFDF91CF911F9196
:100910000F91FF90EF90DF90CF90BF90AF909F909E
:100920008F900895FF920F931F930E94420168EEEB
:1009300073E080E090E00E94D105FF241EC0812F6B
:10094000602F4F2D21E00E94010165E070E080E002
:1009500090E00E94D10564E670E080E090E00E94A3
:10096000D1051F5F183059F70F5F083011F010E004
:10097000E6CFF39488E0F81611F000E0F8CF68EEC7
:1009800073E080E090E00E94D1050E94420183E084
:1009900090E06CEB72E00E94680282E090E06CEB09
:1009A00072E00E94680281E090E06CEB72E00E94CD
:1009B00068020E94FB028BE490E061E070E00E941C
:1009C00028048BE490E060E070E00E94280410E0CE
:1009D00081E060E070E046EB53E022E030E00E940E
:1009E000720381E061E070E046EB53E022E030E02A
:1009F0000E94720382E060E070E046EB53E022E088
:100A000030E00E94720382E061E070E046EB53E068
:100A100022E030E00E94720383E060E070E046EB89
:100A200053E022E030E00E94720383E061E070E076
:100A300046EB53E022E030E00E9472031F5F1A3061
:100A400039F61F910F91FF9008950F931F930AEEAF
:100A500011E0C80140E855E260E070E00E946306E2
:100A600068EE73E080E090E00E94D105C80160E08C
:100A700071E00E948E088FEF84B98CEF8AB915B8A7
:100A80008BB183708BB9E0EBF0E01082A1EBB0E0AA
:100A90001C9280818260808382E38093B3001092F5
:100AA000B2008C9186608C93E0E7F0E080818260F8
:100AB00080831F910F9108950E94F7050E942505DC
:100AC0000E949204FDCF1F920F920FB60F92112435
:100AD0002F933F938F939F93AF93BF938091610127
:100AE00090916201A0916301B09164013091650120
:100AF0000196A11DB11D232F2D5F2D3720F02D57FD
:100B00000196A11DB11D2093650180936101909311
:100B10006201A0936301B093640180915D019091A3
:100B20005E01A0915F01B09160010196A11DB11D10
:100B300080935D0190935E01A0935F01B09360018B
:100B4000BF91AF919F918F913F912F910F900FBEC9
:100B50000F901F9018959FB7F89420915D013091E8
:100B60005E0140915F015091600186B5A89B06C06F
:100B70008F3F21F02F5F3F4F4F4F5F4F9FBF542F4D
:100B8000432F322F2227280F311D411D511D82E096
:100B9000220F331F441F551F8A95D1F7B901CA018F
:100BA0000895EF92FF920F931F93CF93DF937B01F2
:100BB0008C010E94AB05EB010EC00E94AB056C1BC3
:100BC0007D0B685E7340C8F30894E108F1080109E1
:100BD0001109C851DC4FE114F1040105110569F751
:100BE000DF91CF911F910F91FF90EF90089578942E
:100BF00084B5826084BD84B5816084BD85B5826022
:100C000085BD85B5816085BDEEE6F0E080818160BF
:100C10008083E1E8F0E010828081826080838081BF
:100C200081608083E0E8F0E0808181608083E1EB97
:100C3000F0E0808184608083E0EBF0E0808181607F
:100C40008083EAE7F0E08081846080838081826035
:100C5000808380818160808380818068808310921E
:100C6000C10008951F920F920FB60F9211242F9377
:100C70003F934F938F939F93EF93FF934091C600C1
:100C8000E091E601F091E70131969F012F773070F6
:100C900031978091E8019091E9012817390739F0DF
:100CA000EA59FE4F40833093E7012093E601FF911C
:100CB000EF919F918F914F913F912F910F900FBE88
:100CC0000F901F901895CF93DF93EC019A01AB0121
:100CD000E885F985203081EE380780E0480780E01C
:100CE000580709F449C081E090E00A8802C0880FE3
:100CF000991F0A94E2F7808360E079E08DE390E049
:100D00000E94CE082150304040405040CA01B901F5
:100D100022E030E040E050E00E94CE08EC81FD810E
:100D20003083EE81FF812083EA85FB85208141E0CD
:100D300050E0CA010E8402C0880F991F0A94E2F79E
:100D4000282B2083EA85FB852081CA010F8402C0FD
:100D5000880F991F0A94E2F7282B2083EA85FB85E8
:100D60008081088802C0440F551F0A94E2F7842B43
:100D70008083DF91CF910895108220E130E0CECFC3
:100D8000DC011296ED91FC911397E058FF4F2191F1
:100D9000319180819181281B390B2F773070C901E7
:100DA0000895DC011296ED91FC911397EE57FF4FD9
:100DB0002081318192918291E058F040821793070F
:100DC00019F42FEF3FEF05C0E20FF31F8081282FAA
:100DD00030E0C9010895DC011296ED91FC91139762
:100DE000DF01AE57BF4F2D913C911197E058FF4F57
:100DF00080819181E058F0408217930719F42FEF1A
:100E00003FEF0BC0E20FF31F80812F5F3F4F2F7723
:100E100030702D933C93282F30E0C9010895DC01F8
:100E20001296ED91FC911397EE57FF4F80819181BF
:100E3000929382930895FC01A085B18521898C91BC
:100E400090E0022E02C0959587950A94E2F780FF04
:100E5000F6CF0484F585E02D608308958EE091E05F
:100E60009093EB018093EA0186E691E09093ED0187
:100E70008093EC0185EC90E09093EF018093EE017C
:100E800084EC90E09093F1018093F00180EC90E08D
:100E90009093F3018093F20181EC90E09093F5013F
:100EA0008093F40186EC90E09093F7018093F60133
:100EB00084E08093F80183E08093F90187E08093D8
:100EC000FA0185E08093FB0181E08093FC010895A5
:100ED0000F931F93CF93DF938C01EB0109C02196F1
:100EE000D801ED91FC910190F081E02DC8010995A8
:100EF00068816623A1F7DF91CF911F910F9108952B
:100F0000EF92FF920F931F93CF93DF938C017B019E
:100F1000EA010CC0D7016D917D01D801ED91FC91E2
:100F20000190F081E02DC80109952197209791F754
:100F3000DF91CF911F910F91FF90EF900895DC0109
:100F4000ED91FC910280F381E02D099508952F9297
:100F50003F924F925F926F927F928F929F92AF9249
:100F6000BF92CF92DF92EF92FF920F931F93DF9386
:100F7000CF93CDB7DEB7A0970FB6F894DEBF0FBE04
:100F8000CDBF1C016A017B01411551056105710549
:100F900049F440E350E060E070E020E030E00E947F
:100FA000410856C0882499245401422E55246624B1
:100FB000772401E010E00C0F1D1F080D191DC7015B
:100FC000B601A30192010E94AC08F8016083089465
:100FD000811C911CA11CB11CC701B601A301920187
:100FE0000E94AC08C901DA016C017D01C114D10471
:100FF000E104F104F1F681E0E82EF12CEC0EFD1E87
:10100000E80CF91C3E010894611C711CD501C40157
:101010000197A109B1096C01C818D90816C0F601D9
:10102000EE0DFF1D40814A3010F4405D01C0495C67
:10103000552747FD5095652F752FC10120E030E001
:101040000E9441080894E108F1086E147F0439F702
:10105000A0960FB6F894DEBF0FBECDBFCF91DF9143
:101060001F910F91FF90EF90DF90CF90BF90AF90C6
:101070009F908F907F906F905F904F903F902F90B8
:101080000895EF92FF920F931F93CF93DF93EC019C
:101090007A018B012115310541F4E881F981019034
:1010A000F081E02D642F09951BC02A303105B1F481
:1010B00077FF10C04DE250E060E070E020E030E0EB
:1010C0000E94410810950095F094E094E11CF11CF9
:1010D000011D111DCE01B801A7012AE00E94A7073A
:1010E000DF91CF911F910F91FF90EF9008950F9393
:1010F0001F938C014DE050E060E070E020E030E0B4
:101100000E944108C8014AE050E060E070E020E041
:1011100030E00E9441081F910F9108950F931F9393
:101120008C010E949F07C8010E9477081F910F91B0
:10113000089597FB092E07260AD077FD04D049D0E1
:1011400006D000201AF4709561957F4F0895F6F748
:10115000909581959F4F0895A1E21A2EAA1BBB1B63
:10116000FD010DC0AA1FBB1FEE1FFF1FA217B30773
:10117000E407F50720F0A21BB30BE40BF50B661F89
:10118000771F881F991F1A9469F76095709580954D
:1011900090959B01AC01BD01CF01089597FB092EED
:1011A00005260ED057FD04D0D7DF0AD0001C38F436
:1011B00050954095309521953F4F4F4F5F4F089583
:1011C000F6F790958095709561957F4F8F4F9F4F63
:1011D0000895AA1BBB1B51E107C0AA1FBB1FA6177E
:1011E000B70710F0A61BB70B881F991F5A95A9F7D0
:1011F00080959095BC01CD0108952F923F924F921A
:101200005F926F927F928F929F92AF92BF92CF9296
:10121000DF92EF92FF920F931F93CF93DF93CDB79F
:10122000DEB7CA1BDB0B0FB6F894DEBF0FBECDBF17
:1012300009942A88398848885F846E847D848C84E8
:101240009B84AA84B984C884DF80EE80FD800C81F1
:101250001B81AA81B981CE0FD11D0FB6F894DEBFD4
:101260000FBECDBFED010895EE0FFF1F0590F49165
:10127000E02D0994A0E0B0E0E0E4F9E00C94050969
:10128000EC01A880B980CA80DB80A114B104C1043C
:10129000D10441F484E2A82E89EDB82E8BE5C82E46
:1012A00087E0D82EC601B5012DE133EF41E050E0D3
:1012B0000E94CE0827EA31E440E050E00E949B09FA
:1012C0007B018C01C601B5012DE133EF41E050E017
:1012D0000E94CE08CA01B9012CEE34EF4FEF5FEF48
:1012E0000E949B096E0D7F1D801F911F97FF04C0F8
:1012F0006150704080409048688379838A839B83E3
:101300009B013F77C901CDB7DEB7EAE00C94210914
:101310000E943A09089586E091E00E943A090895F2
:10132000A0E0B0E08093060190930701A09308012C
:10133000B09309010895629FD001739FF001829FCD
:10134000E00DF11D649FE00DF11D929FF00D839F54
:10135000F00D749FF00D659FF00D9927729FB00DF1
:10136000E11DF91F639FB00DE11DF91FBD01CF0104
:0813700011240895F894FFCF49
:10137800626567696E0001000000000000001B073D
:0C13880068078007C006EB06D1060F07BF
:00000001FF
